:100000000C942A000C9445000C9445000C94450077
:100010000C9445000C9445000C9445000C9445004C
:100020000C9445000C9445000C9445000C9445003C
:100030000C9445000C9445000C9445000C9445002C
:100040000C9445000C9445000C9445000C9445001C
:100050000C94450011241FBECFE5D4E0DEBFCDBF18
:1000600010E0A0E6B0E0E2ECF1E002C005900D92F5
:10007000A036B107D9F710E0A0E6B0E001C01D92AC
:10008000A036B107E1F70C94CC000C940000CF939C
:10009000DF93CDB7DEB781E0809338001092350052
:1000A0001092320081E08093370010923400109259
:1000B0003100DF91CF910895CF93DF93CDB7DEB7B5
:1000C00025970FB6F894DEBF0FBECDBF8983898117
:1000D000282F33273D832C838C819D81813091058E
:1000E000B9F02C813D81223031052CF48C819D8129
:1000F000009739F035C02C813D812230310571F0F7
:100100002FC08EEF909138008923809338003BC038
:100110008091380081608093380035C09EEF8091D7
:10012000380089238093380080E29EE49B838A8391
:100130008A819B81009731F08A819B8101979B8303
:100140008A83F6CF8091380081708093380080E2F6
:10015000898389818823B9F0898181508983F9CF86
:1001600080913600992781709070009739F08EEF5A
:100170009091380089238093380005C08091380021
:1001800081608093380025960FB6F894DEBF0FBECD
:10019000CDBFDF91CF910895CFE5D4E0DEBFCDBFD5
:1001A0000E944700809136009927807190700097D7
:1001B00021F081E00E945C00F5CF80E00E945C00AD
:0201C000F1CF7D
:00000001FF
